:020000020000FC
:1000000012C0189518951895189518951895189563
:10001000BAC7C0C7189518951895189518951895CA
:100020001895189518950FE50DBF04E00EBF0FE069
:1000300008BB0EEE07BB0FE105BB00E204BB0FE7F8
:1000400002BB00E801BB02E371D79899FFCFAD9ADC
:10005000979A07EC07B907E006B900E805BF00E882
:1000600008B902E50DB9B4D3BAD3A7D3FF93EF9380
:10007000E653F140EF91FF9128F400E50DB901E05E
:10008000002E13C200270093600003B30F710631E6
:10009000C9F405E04BD703B30F71063199F403B3EC
:1000A0000F710F31E1F701E0009377000027009313
:1000B0007C0000937D000093A70200937E000093D4
:1000C0007F0035C0E0E0F0E047D710937700EAE02A
:1000D000F0E042D71093A702E1E0F0E03DD71093A3
:1000E0007C00E2E0F0E038D710937D00E3E0F0E040
:1000F00033D710937E00E4E0F0E02ED710937F001A
:10010000E5E0F0E029D710937800E6E0F0E024D7AE
:1001100010937900E7E0F0E01FD710937A00E9E050
:10012000F0E01AD7133008F0112710936000E8E0D0
:10013000F0E012D71B3818F4123108F001C012E4B5
:100140001093A0020AE00093A50200E00093A4022D
:100150000093A60203B30F710F31E1F72AE0A9D68D
:100160002A95E9F7C29800E000936D0000E0009343
:100170006E0000E000936F0000E00093700000E06C
:1001800000937100A0D61F3F59F0113019F00AE01A
:10019000C5D6F8CF01E000936D0095D61130E9F394
:1001A000C29A00E50DB91F3F19F402E0002E7DC18F
:1001B00067D5112319F003E0002E77C10FEF8AD421
:1001C000662309F0CAD31091A902112371F460913A
:1001D000A802662339F001E0162FF4D4112329F484
:1001E0006A95C9F704E0002E60C1009177000023F2
:1001F00009F42BC01091A702112339F06091A802D5
:10020000662319F10FEFDED402C004E163D4112399
:10021000E1F010937600D2D3009177001091A702FD
:10022000F7D3112392F000919C00109178000117F0
:1002300061F400919D0010917900011731F4009153
:100240009E0010917A000117E9F001E00093770019
:10025000112710937C0010937D002091A902222386
:1002600021F01093A70236D40AC061E06093A70280
:100270000FEF162FA7D4112311F46395F7CF109326
:1002800076009CD39AD2FF93EF93EC57F140EF9115
:10029000FF9110F003E011C0FF93EF93E856F14097
:1002A000EF91FF9110F002E008C0FF93EF93E45547
:1002B000F140EF91FF9150F001E0002E979804E695
:1002C00035D6979A04E632D60A94C1F700917700A2
:1002D00010917600101798F501E0009377003091A7
:1002E0006000332339F04091A2024D3119F0403FB4
:1002F00009F025C01091A70213950091A8020117DB
:1003000008F407C01093A7020FEF5CD4112391F3F8
:1003100013C011271093A7024091A2024D3119F08A
:10032000403F09F072C044274093A2021091A902F5
:10033000112301F304E1CED3109376003FD3442779
:100340004093A202B7D0F89400E00EBD1123C1F093
:100350001AF405E0002EA9C011241394012C79D2BF
:100360004091A2024D3181F04B31F9F0403FB9F09C
:10037000403EF9F04E3119F000917700E0CF45C0D2
:1003800000916000023029F00091770003950093FE
:100390007700112710937C0010937D0073CF00919C
:1003A0007600039500937700F4CF109177001A95AB
:1003B00021F51091A702112359F01A9569F41091B3
:1003C000A902112329F011271093A70283D30BC090
:1003D0001091A802112399F31093A7020FEFF2D303
:1003E000112309F4EACF10937600E8D21091760039
:1003F0000091A202003E09F411E01093770011274A
:1004000010937C0010937D003DCFF894009177000D
:10041000E0E0F0E095D50091A702EAE0F0E090D5A9
:100420000A2DE1E0F0E08CD50B2DE2E0F0E088D57C
:1004300000916800039503191127080D911EE3E050
:10044000F0E07ED5092DE4E0F0E07AD50091780067
:10045000E5E0F0E075D500917900E6E0F0E070D5D8
:1004600000917A00E7E0F0E06BD50091A002E8E0AF
:10047000F0E066D500916000E9E0F0E061D510E0C1
:1004800020E030E1C2D108EC51D5979803B30F7149
:100490000F31E1F70AEF4AD511E0C4D111E038601D
:1004A000B4D1C798AD988895FFCFF89411241394D0
:1004B000D0D1E5CF009177001091A702A9D21123E6
:1004C00022F000918B00003211F011270895C090A6
:1004D0009C00D0909D00E0909E00F0909F00FF2037
:1004E00011F010E00895C0927800D0927900E09267
:1004F0007A00A0909A00B0909B0022271E2D0D2D0F
:100500001695079508F421E0802E912E6C2C722E02
:1005100030906800A0909A00B0909B0000917C0001
:1005200010917D002227202B212B49F4A0927C00E2
:10053000B0927D0080927E0090927F0006C0A02E37
:10054000B12E80907E0090907F000A2D0B210F3FEE
:1005500029F0BB2029F402E0A01610F41EEF089544
:1005600092D13DD100270093A3020093A10201E0A4
:100570001127801A910A08F434C0F0926E00E092BC
:100580006F00D0927000C0927100D9D1C0EAD0E063
:10059000B09905C048D04423DAF3142F0895099187
:1005A000C6988DD4C69AC03A99F7D23089F73A9452
:1005B00031F002E01127D00EE11EF11ED8CF7AD122
:1005C000A42CB52C0A2D0B210F3F29F0BB2029F4B8
:1005D00002E0A01610F41EEF08953090680053D189
:1005E000C6CF062D072911F411270895F0926E0049
:1005F000E0926F00D0927000C0927100A0D1C0EA6A
:10060000D0E06C0E7D1EB09905C00DD04423DAF306
:10061000142F08950991C69852D4C69AC615D705C5
:1006200090F311270895F89400E00EBDE091A40224
:10063000F091A502319729F0E093A402F093A5026E
:1006400020C000E00093A4020AE00093A502B5D008
:10065000FF93EF93E153F140EF91FF9190F401E0AC
:1006600065D4ABD0FF93EF93E153F140EF91FF914D
:1006700040F40AE0002E1124ECD00EE10093A20217
:1006800058C033B33F713F3121F00091A1020317ED
:1006900031F03093A10200270093A30240C03091B3
:1006A000A3023395373019F03093A30238C000937A
:1006B000A20233273093A1023093A302073139F409
:1006C0002091A0022450223128F522E123C00F30CE
:1006D00039F42091A0022C5F2A38E0F02AE81AC0F1
:1006E0000D3159F40AEF22D433B33F713D3119F47F
:1006F00000EF0093A20241E01EC00B3131F50AEF7A
:1007000015D433B33F713B3119F400EE0093A202CC
:1007100042E011C02093A0021BE0322F76D000E20D
:1007200009BF00E40EBDB09902C0789488954FEFE0
:1007300002C043E0089500E80DBD00E00CBD04E0F8
:1007400009BF04E00EBD789408950E3141F708EC1E
:10075000EDD333B33F713E3161F306E4E7D300E0FC
:1007600002BF01E009BF05E003BF789433B33F71D6
:10077000373181F404E6DAD333B33F71373151F4C2
:10078000009160000A950AF402E00093600044279B
:100790004093A60233B33F713E3141F702E3C6D323
:1007A00033B33F713E3111F733B33F713F31E1F75E
:1007B000979AF89400E003BFBACF379A349A369AE2
:1007C000349BFECFE4B1F5B13798F695E7950895DF
:1007D000C79A0FE0ABD3C69AB09BFECF08953327DC
:1007E000EEE7FFE02CD03395D9F710E028E034E0B5
:1007F0000CD0B09BFECF13E028E930E006D01BE020
:100800002091A002322F01D00895C19802E057D361
:10081000012F55D3022F53D3032F51D3C19A0AE08E
:100820007DD30895C19803E04AD3012F48D341D323
:10083000212F3FD3312FC19A0AE070D3089558E099
:10084000B09BFECFC69805913AD3C69A5A95C1F788
:100850000895C5DF10E028E030E2D7DF04E666D374
:10086000112019F0E6E6FFE002C0EEE6FFE0E7DF68
:1008700004E65CD3E6E7FFE0E2DF0EE157D30A943B
:1008800079F7ADDF0895CC24D0906200E09063004A
:10089000F09064000A2D1B2D025010402227039D6A
:1008A000D00CE11CF21E139DE00CF11CDD0CEE1CC3
:1008B000FF1C089500271091690020916A003327DA
:1008C000110F221F331FCA2CDB2CEE24CC0CDD1C95
:1008D000EE1CFF240C0D1D1D2E1D3F1DEFEFF1E042
:1008E000E023F12300271E7F30936E0020936F00DA
:1008F0001093700000937100B3D2112321F0CED277
:10090000442455240895A0E0B0E0D3D2AE17BF0729
:1009100019F0CFD21296F9CF212FCBD2312F3F3FF2
:1009200021F4273F10F03FEF2FEF422E532E129667
:10093000B23019F0BED2BDD2FACFB0D2089590D263
:10094000112309F00895C0EAD0E0B3D21993C03A58
:10095000E1F7D230D1F7A2D20895AAEAB2E0002797
:100960000D93A63CE9F7B230D9F7EAEDF2E04091F9
:10097000A8026091A802552702811381CAEDD2E036
:100980002A813B813117200708F453956A9511F0AD
:100990002496F6CFAAEAB2E0550F0027A50FB01FA4
:1009A0000D911D91012BE1F71297008111810D939B
:1009B0001C934A9511F03496DCCF0895A6ECB2E072
:1009C0000FEF0D93AA3DE9F7B230D9F7EAEDF2E067
:1009D000452F652F772701811281CAEDD2E0298149
:1009E0003A813117200708F473956A9511F0239620
:1009F000F6CFA6ECB2E00027A70FB01F0D910F3F76
:100A0000E9F700810E934A9511F03396E2CF0895ED
:100A1000053130F4002321F02091A802211710F4B1
:100A20001FEF08950A952227A6ECB2E0A00FB21F8F
:100A30002C916627220F661F2295022F0F70629558
:100A4000602B207F422F51E056236E7F1123F9F057
:100A5000110F0027E8EAF2E0E10FF01FA190B0804B
:100A60000A2D0B210F3F19F00A2D0B2911F41FEF4E
:100A7000089530906800330C762F731920F01ADF38
:100A8000A42CB52CFACF30906800FDDE09C0CC2430
:100A9000D0906600E0906700FF24DD0CEE1CFF1C88
:100AA000D60EEC1CFC1CF0926E00E0926F00D0920F
:100AB0007000C092710043DFC0EAD0E0C40FD51FC0
:100AC000A0E8B0E009910D93A03AE1F7B030D1F77A
:100AD00011270895402F55276627CC24D090660013
:100AE000E0906700FF24DD0CEE1CFF1CF0926E000E
:100AF000E0926F00D0927000C092710077271FDFE4
:100B0000C0EAD0E00881002309F453C0053EE1F1BA
:100B10000A8D1B8D012BC1F10B8510E11023B9F05B
:100B20004F3F91F56395AAEDB2E00027162F1A9575
:100B3000110F110FA10FB01F0A8D0D930B8D0D9387
:100B400008810D9309810C936E30F1F432C000726C
:100B5000D9F008850D34C1F409850035A9F40A855A
:100B6000033391F453954F3F69F0AAEDB2E003E0EF
:100B7000152F1A95019FA00DB11D7D9308810D932E
:100B800009810C935431A9F0739599F0A096C03A5D
:100B900009F0B8CFD23009F0B5CF02E01127D00E5E
:100BA000E11EF11EF0926E00E0926F00D092700094
:100BB000A6CF4F3F21F4A8EAB2E06D935C93042FD7
:100BC000152F0895402F77275527110FE8EAF2E0F7
:100BD000E10FF51FA190B0800FEF0B210A210F3F0D
:100BE00009F40895309068004EDEF0926E00E092B5
:100BF0006F00D0927000C0927100A1DEC0EAD0E018
:100C000008810023D1F1053E11F10A8D1B8D012BC6
:100C1000F1F00B850072D9F008850D34C1F4098517
:100C20000035A9F40A85033391F45395451729F14A
:100C3000AAEDB2E003E0152F1A95019FA00DB11D9A
:100C40007D9308810D9309810C935431B1F0739514
:100C5000A1F0A096C03AA1F6D23091F63A9431F0C4
:100C600002E01127D00EE11EF11EBFCF23DE2323A9
:100C70002F3F19F0A42CB52CB5CF042F152F0895B4
:100C800000E00093720000E00093730001E0009325
:100C900074000EEB00937500B4D020908800309063
:100CA00089000027122D232D3327110F221F331FF8
:100CB00030937200209373001093740000937500BA
:100CC000A0D000918B0010918C001F930F930050C7
:100CD00012400F911F9111F012E0089500918D00C4
:100CE0000093680000918E0010918F00020D131D7B
:100CF0000093690010936A00009191001091920096
:100D000000936B0010936C00A0909600B090970039
:100D1000AA2021F4BB2011F411E008952091900045
:100D2000A29E112D002DB29E100D209169003091D0
:100D30006A00020F131F0093660010936700009172
:100D40006B0010916C001295212F207F1F703FE0E7
:100D5000302302950F70022B332311F00F5F1F4FCA
:100D6000209166003091670000241124200F311F6C
:100D7000011C209362003093630000926400109283
:100D80006500009193001091940022273327FF24DF
:100D9000F12AF02AB1F400E2FF24220C331CFF1CDC
:100DA000F0927200309273002092740000937500EC
:100DB00028D0009180001091810020918200309114
:100DC0008300D0906900E0906A00FF240D191E098D
:100DD0002F093F09442750916800652F5295507F95
:100DE00062956F707727041715072607370712F0EB
:100DF00001E003C0002713E008950093610011276C
:100E00000895F0907200E0907300D0907400C0904C
:100E100075003F2D2E2D1EEF1D21002730936E00F3
:100E200020936F00109370000093710019D011236C
:100E300009F008952C2D31E03D21CC27DD27A0E8D5
:100E4000B0E0E0EAF0E035D0C217D30722F0AE17E9
:100E5000BF070AF41D932196D230A9F71FD0089539
:100E600034E6C29801E100936D002DD0112351F4B6
:100E7000A0E0B0E11ED01E3F11F411270895119794
:100E8000C9F704C01E3F11F411270895C29A04E166
:100E900045D03A9509F0E5CF11E008950AD009D080
:100EA000C8EED7E006D01F3F11F02197D9F7C29ABC
:100EB00008950FEF0FB9779BFECF1FB108950FB9BB
:100EC000779BFECF0895C8EED7E0F3DF1F3F21F0F8
:100ED0002197D9F711E0089500916D00102F00645B
:100EE000EEDF00916E00EBDF00916F00E8DF009114
:100EF0007000E5DF00917100E2DF112311F405E9D4
:100F000001C001E0DCDFC8EED7E0D3DF1E3F29F0EF
:100F100020E8212311F02197C1F708950000000077
:100F20000000000000000A95C9F7089514E623E1C7
:100F300000002A95E9F71A95D1F70A95B9F70895AF
:100F40000BD0011709F40895E199FECFFFBBEEBB6A
:100F50000DBBE29AE19A0895E199FECFFFBBEEBB8B
:100F6000E09A1DB3089553EF6EF00000000053EFB8
:100F70006EE8000000004578697400000000000081
:100F80000000000000000FE50DBF04E00EBF00E010
:100F90000EBD5BC90FB6E0916000F5E0EA9512F076
:100FA000FF0FFCCF4091A60243954F1731F4442721
:100FB000979902C0979A01C097984093A6020FBED6
:020FC000189582
:00000001FF
